:020000040000FA
:020000002728AF
:08000800940B0A28950B0A284D
:1000100010120612920B0F2813140B110900131063
:100020000B11090013181B28051E12280508910042
:1000300011120311080003150800051A1D280800F5
:1000400044309200080010309500940108002030E0
:10005000830086011F308500873081000301830003
:100060008601061490019301A0308B001D2086129A
:10007000930112200B30110203193F28362820204B
:1000800086161D2012200319362805301102031987
:100090004A287D281D201220031936281D2011080A
:1000A00082073628652869286D28712873287528E5
:1000B000772879287C28612836283628362836285B
:1000C0003628F030900510147D28F03090059014FB
:1000D0007D28F030900590157D28F03090051015A2
:1000E0007D2890177D2890137D2810177D281013E8
:1000F0007D28101623207D2810121220031936287F
:100100000C301102031986281D207D281D2010089F
:10011000860036282834433429344734573436345B
:060120004234573458344C
:00000001FF
